:02000000142AC0
:0800080021088A0182070C1097
:100010008C1D0129190840398C110319012900167A
:10002000A01DA00C0512201E00128E01F6308F00BC
:100030003C300C108E00163000298C1D3128190818
:1000400040398C11031931280016A01DA00C05128F
:10005000201E00128E01F6308F003C300C108E00F6
:1000600001290C1C01290C100016A01DA00C051262
:10007000201E00128E01FB308F001E300C108E00EF
:100080003B3000298C1D5128190840398C11031967
:1000900051288E01F6308F003C300C108E00163047
:1000A00000290C1C01290C104F3000290C108C1D4C
:1000B0000129190840398C11031901290016A01DC6
:1000C000A00C0512201E00128E01F2308F00543059
:1000D0000C108E002008A6002408A7006930002913
:1000E0008C1D8528190840398C11031985280016A4
:1000F000A01DA00C0512201E00128E01F6308F00EC
:100100003C300C108E00163000290C1C01290C10FC
:040110004F30002943
:10020000A10022088A0A82070B1C022A0508083965
:100210000B100319022A230981018B160B1181008F
:100220000230A4001030012A0B1C442905080839AB
:100230000B1003194429A51937290016A01EA00D7B
:100240000516201E0012A412A40A230981018B1690
:100250000B11810024183329A519A30AA51C3329E1
:10026000A30B3329A5019B30A41E1030012AA41230
:10027000A40AA501A301230981018B160B1181009A
:100280009B30A41E1030012A0B1D022A8B1200166F
:10029000A01EA00D0516201E0012A412A40A2308F9
:1002A000163E81018B160B1181005330012A0B1C65
:1002B0008429050808390B10031984292518722987
:1002C000230981018B160B11810024186E29A519B1
:1002D000A30AA51C6E29A30B6E29A5019B30A41EA1
:1002E0001030012AA50A0016A01EA00D0516201E1A
:1002F00000129B30A300230981018B160B11810092
:100300009B30A41E1030012A0B1D022A8B120016EE
:10031000A01EA00D0516201E00120230A4008D3074
:10032000012A0B1C022A050808390B100319022A9E
:10033000230981018B160B1181001030012A0B1C3F
:10034000B529050808390B100319B5290016A01E98
:10035000A00D0516201E00120230A4002309810101
:100360008B160B1181001030012A0B1D022A8B12F3
:100370000016A01EA00D0516201E00120130A400BC
:10038000643081018B160B118100C330012A0B1CD4
:10039000DD29050808390B100319DD290016A01EF8
:1003A000A00D0516201E00120230A40023098101B1
:1003B0008B160B1181001030012A0B1D022A8B12A3
:1003C0000016A01EA00D0516201E00120230A4006B
:1003D000E630012A0B1C022A050808390B10031904
:1003E000022A230981018B160B1181002418FF2991
:1003F000A519A30AA51CFF29A30BFF29A5011030ED
:10040000012AA2002508031D09002708A619013E9C
:10041000FD3E1F390319090010390319112AA515CA
:10042000090025152514090085018316FF23900076
:1004300003309F001B308500083096008330810018
:1004400009308C0083120130990048308B00013054
:100450009000853084001030A000A101A201A50108
:10046000A301A4018F01190805088C110B100C10B1
:0604700000008B173A2A80
:02400E0084012B
:00000001FF
